:100000000C948E000C949E110C94AB000C94AB00DD
:100010000C94AB000C94AB000C94AB000C94AB00B4
:100020000C94AB000C94AB000C94AB000C94AB00A4
:100030000C94AB000C94AB000C94AB000C94AB0094
:100040000C94AB000C94AB000C94AB000C94AB0084
:100050000C94AB000C94AB000C94AB000C94AB0074
:100060000C94AB000C94AB001201100100000008CE
:100070005E040202000100000001090220000101EB
:100080000080320904000002584200000705820384
:1000900020000407050203080004FF0004FF060710
:1000A00005FF020103FFFFFFFFFFFF0206FF04033E
:1000B00005FF000107FFFFFF00020104FF03FF0629
:1000C00007FFFF05040309042A0377007700770080
:1000D0002E006200720075006E006F0066007200F4
:1000E000650069007400610073002E0063006F00FA
:1000F0006D002A03550053004200200052006500A5
:10010000740072006F005000610064002000410024
:1001100064006100700074006500720011241FBE4D
:10012000CFEFD4E0DEBFCDBF11E0A0E0B1E0EAEB5D
:10013000F6E202C005900D92A230B107D9F711E0A6
:10014000A2E0B1E001C01D92A23DB107E1F70E941B
:1001500070050C945B130C9400000F931F93FF9396
:10016000EF93BF93AF93F92FE82F09E00093590164
:1001700000E200935A0100E000935B0101E000936C
:100180005C0101E000935D0100E000935E010093DB
:100190005F010093600109E20093610107D0BF9104
:1001A000AF91EF91FF911F910F910895A1E0B9E5F3
:1001B00009E02D980000000000002C9800000000CD
:1001C00000002C9A000000002C98000000000000A5
:1001D0002C9A0000000000002C9800000000000095
:1001E0002C9A0000000000002C9800000000000085
:1001F0002C9A00000000000000002D9A1D9117FDB0
:100200002C9A17FF2C982D98000000002C9A16FDB0
:100210002D9A16FF2D982C9A000000002D9A15FD9E
:100220002C9A15FF2C982D9A000000002C9A14FD92
:100230002D9A14FF2D982C9A000000002D9A15FD80
:100240002C9A15FF2C982D9A000000002C9A14FD72
:100250002D9A14FF2D982C9A000000002D9A15FD60
:100260002C9A15FF2C982D9A000000002C9A14FD52
:100270002D9A14FF2D982C9A000000002D9A0A95B3
:100280002D9A2C9A0895F92FE82F21E030E0E20F03
:10029000F31F2227332744275527662777278827E8
:1002A000992790E099D0B6D082D0292F80D0392FCD
:1002B0007ED0492F253021F0293089F180E0089542
:1002C000BFEFBA95F1F7B8ECBA95F1F791E084D0A9
:1002D000A1D06DD0292F6BD0392F69D0492F67D08D
:1002E000592F40835195518340E050E027FD4160F4
:1002F00026FD426025FD526024FD51602F7035FDC2
:10030000406434FD406833FD446032FD486031FD97
:10031000406130FD406245835683822F0895B4E6E4
:10032000BA95F1F790E458D093E056D092E054D0CB
:1003300071D03DD0292F3BD0392F39D0492F37D01C
:10034000592F35D0692F33D0792F31D0892F2FD025
:10035000405850585195408351836058619570586A
:1003600071956283738340E050E020FD416021FD80
:10037000426022FD486023FD406124FD516034FD50
:10038000526035FD406836FD4064803408F04064BA
:10039000903408F04068458356833F70232F3E7F9A
:1003A00031FD31603D7F20FD3260832F089590E064
:1003B000B4E1A8E0BA9579F01899FCCFB9E0BA9504
:1003C000F1F7990F18999160B4E1BA9521F0189B53
:1003D000FCCFAA9579F70895A8E097FD0DC0209A63
:1003E000BDE0BA95F1F700002098B3E0BA95F1F7B7
:1003F000990FAA9591F70895209AB3E0BA95F1F76D
:10040000000000002098BDE0BA95F1F7990FAA9579
:1004100021F70895209AB3E0BA95F1F700000000A3
:1004200020980895A8950895FC01808190E0807639
:1004300090708032910559F481818130E1F483E339
:1004400091E0909394018093930184E10895803426
:10045000910589F48181863071F481E090E0909378
:1004600003018093020187E491E0909394018093CB
:10047000930180E1089580E00895809102019091B8
:1004800003010895CF93DF938091AF0186FD07C0EC
:10049000CFEAD1E00E942C10888186FFFBCF83E356
:1004A00091E064E10E947B11DF91CF910895E3E335
:1004B000F1E084E2DF011D928A95E9F794E19183EE
:1004C00080E1848B82E4858B168A81E0878B808F24
:1004D00082E0818F928F86E0838F7C962FEF87E575
:1004E00091E02193E817F907E1F708950F931F931F
:1004F0008C010E945702012B61F02FE088E190E00F
:100500000FB6F894A895809360000FBE209360000A
:1005100008C088E10FB6F8948093600010926000E4
:100520000FBE0E941510F894EAE2F0E0808182602C
:10053000808380818660808326EF39E047E751E041
:10054000CA010197F1F721503040D1F7EAE2F0E01B
:1005500080818D7F80838081897F808378941F91C3
:100560000F9108952F923F924F925F926F927F92D8
:100570008F929F92AF92BF92CF92DF92EF92FF92B3
:100580000F931F93DF93CF93CDB7DEB73B014C01A1
:1005900019012A016D897E898F89988D6A197B09D5
:1005A0008C099D09621A730A840A950AA4019301B1
:1005B0000E94FF12E218F30804091509A801970127
:1005C0000E941E132A0D3B1D4C1D5D1D622F732FB3
:1005D000842F952FCF91DF911F910F91FF90EF9076
:1005E000DF90CF90BF90AF909F908F907F906F9053
:1005F0005F904F903F902F9008951AB889EF8BB974
:1006000014B88FE385B917B888B908952F923F922F
:100610004F925F926F927F928F929F92AF92BF9212
:10062000CF92DF92EF92FF920F931F93CF93DF93BE
:10063000EC01DB018D8180FF06C0E5E3F1E0808104
:100640008160808305C0E5E3F1E080818E7F808357
:100650008D8182FF06C0E5E3F1E0808182608083C6
:1006600005C0E5E3F1E080818D7F80838D8183FF8C
:1006700006C0E5E3F1E080818460808305C0E5E3A6
:10068000F1E080818B7F80838D8181FF06C0E5E36F
:10069000F1E080818860808305C0E5E3F1E080813E
:1006A000877F80838F8183FF06C0E5E3F1E080814F
:1006B0008061808305C0E5E3F1E080818F7E8083E7
:1006C0008F8182FF06C0E5E3F1E080818062808354
:1006D00005C0E5E3F1E080818F7D80838F8180FF1D
:1006E00006C0E5E3F1E080818064808305C0E5E336
:1006F000F1E080818F7B80838F8181FF06C0E5E3FD
:10070000F1E080818068808305C0E5E3F1E08081CD
:100710008F7780838E8180FD02C080E001C08FEFE3
:10072000809337018E8181FD02C080E001C08FEF90
:10073000809339018E8182FD02C080E001C08FEF7D
:1007400080933A018E8183FD02C080E001C08FEF6B
:10075000809338018E8184FD02C080E001C08FEF5C
:1007600080933D018E8185FD02C080E001C08FEF46
:1007700080933E018E8187FD02C080E001C08FEF33
:1007800080933B018E8186FD02C080E001C08FEF27
:1007900080933C018C91882311F08093370112964D
:1007A0008C911297882311F08093390113968C91C4
:1007B0001397882311F080933A0111968C91119729
:1007C000882311F08093380114968C911497882314
:1007D00011F080933D0115968C911597882311F0A7
:1007E00080933E0116968C911697882311F0809382
:1007F0003B0117966C91662311F060933C0100D089
:1008000000D0EDB7FEB73196698170E080E090E0EE
:100810002FEF3FE740E050E0208331834283538352
:1008200020E83FEF4FEF5FEF0F2EFFE7EF2EF0E0F6
:10083000FF2EF0E00F2FF0E01F2FF02D0F2EF0E035
:10084000AF2EF0E8BF2EFFEFCF2EFFEFDF2EF02D03
:100850000E94B2020F2EFFE36F2EF1E07F2EF02DEB
:10086000F301619371934F01EDB7FEB731966A8141
:1008700070E080E090E00F2EF0E02F2EF0E83F2EA9
:10088000FFEF4F2EFFEF5F2EF02D2082318242824C
:10089000538220E83FEF4FEF5FEF0F2EFFEFAF2EB9
:1008A000FFE7BF2EF0E0CF2EF0E0DF2EF02D0E940C
:1008B000B202F40171836083EDB7FEB731966B81AC
:1008C00070E080E090E0A082B182C282D38220E812
:1008D0003FEF4FEF5FEF0F2EF0E0AF2EF0E8BF2EAF
:1008E000FFEFCF2EFFEFDF2EF02D0E94B202F301BB
:1008F000349671836083EDB7FEB731966C8170E0FA
:1009000080E090E0208231824282538220E83FEFF3
:100910004FEF5FEF0F2EFFEFAF2EFFE7BF2EF0E0A0
:10092000CF2EF0E0DF2EF02D0E94B2020F900F903C
:100930000F900F9026E030E0620E731EF30171837A
:100940006083DF91CF911F910F91FF90EF90DF9027
:10095000CF90BF90AF909F908F907F906F905F905F
:100960004F903F902F900895682FA4E0B1E0E9E107
:10097000F1E088E001900D928150E1F7609304016D
:10098000ACE0B1E0E1E2F1E085E001900D92815050
:10099000E1F760930C01A1E1B1E0E6E2F1E088E06B
:1009A00001900D928150E1F735995BC0349952C0A6
:1009B00086B190E08E7190708430910521F1853080
:1009C000910534F4009771F0029709F056C00FC0FA
:1009D0008830910511F18A309105D1F0069709F020
:1009E0004CC00CC084E091E00E94D60D5CC084E055
:1009F00091E061E171E00E94B60C55C084E091E0A5
:100A00000E94960850C084E091E00E94700938C0AE
:100A100084E091E00E94290846C083B190E086708E
:100A200090708230910589F08630910521F0892BF4
:100A300039F081E023C084E091E00E947D0733C05B
:100A400084E091E00E940F072EC084E091E00E94B4
:100A50009B0929C0339914C084E091E00E94910F52
:100A600022C0339905C084E091E00E94CD051BC0EF
:100A700084E091E00E94B80A03C080E0882399F4E2
:100A800089B1897061F44C9B05C084E091E00E94BB
:100A90009B0509C084E091E00E94650B04C084E0DE
:100AA00091E00E94E809E8E6F0E080818E7F808393
:100AB0000895CF93DF9381E090E00E947602CCE727
:100AC000D2E907C00E941202CE010197F1F70E94FD
:100AD00042020E943D02892BA9F3DF91CF91089534
:100AE0000F931F93CF93DF930E94FD020E9459053D
:100AF00081E00E94B40404E011E0C1E1D1E00E9471
:100B0000120281E00E94B404C801BE010E940603E3
:100B10000E944202F4CFE4E2F0E02081277F2083AC
:100B2000208120632083E5E2F0E020812863208398
:100B30000E94AD000895CF93DF93EC01E5E2F0E071
:100B400080818E7F8083E4E2F0E080818E7F8083ED
:100B5000EBE2F0E080818F778083EAE2F0E0808151
:100B600080688083CE010E944301282F83FF03C049
:100B70008D8181608D8322FF03C08D8184608D8390
:100B800021FF03C08D8188608D8320FF03C08D818C
:100B900082608D83DF91CF910895DC01EAE2F0E07D
:100BA00080818E7E8083EBE2F0E0808181618083B2
:100BB000E4E2F0E080818863808380818D7F8083A0
:100BC000E5E2F0E0808182608083E7E2F0E080810E
:100BD000807E8083E8E2F0E080818F618083489BA3
:100BE0000BC0E4E2F0E0808184608083E5E2F0E025
:100BF0008081837C808314C0E4E2F0E080818B7F7D
:100C00008083E5E2F0E080818C638083E7E2F0E0BE
:100C100080818E7F8083E8E2F0E080818160808344
:100C200087E180937E00EAE7F0E085E0808384E658
:100C300080937C00808180688083808186FDFDCFE9
:100C4000613009F5EAE7F0E080818064808380818B
:100C500086FDFDCF909179008FE7891B12968C93CA
:100C6000129782E680937C00EAE7F0E0808180645E
:100C70008083808186FDFDCF909179008FE7891B6D
:100C800011968C931197E9E2F0E0808110927A003E
:100C900010927E00808180FF17C04C9909C061309E
:100CA00039F416968C911697816016968C93169748
:100CB000199998C0623009F095C016968C911697D4
:100CC000816016968C930895E5E2F0E08081877F3D
:100CD000808385E08A95F1F7309907C016968C914C
:100CE0001697826016968C9316971A9907C01696D7
:100CF0008C911697806116968C931697199907C058
:100D000016968C911697806816968C9316974C9928
:100D100007C017968C911797846017968C93179736
:100D2000E5E2F0E080818860808380818F7E80832F
:100D300085E08A95F1F7309907C016968C91169741
:100D4000846016968C9316971A9907C016968C9104
:100D50001697806216968C931697199907C0179666
:100D60008C911797816017968C9317974C9907C0B1
:100D700016968C911697816016968C931697E5E2DD
:100D8000F0E080818061808380818F7D808385E039
:100D90008A95F1F7309907C016968C91169788605E
:100DA00016968C9316971A9907C016968C911697DB
:100DB000806416968C931697199907C017968C9194
:100DC0001797826017968C9317974C9906C01796C1
:100DD0008C911797886017968C93E5E2F0E08081FC
:100DE00080628083089590E020E0A3E2B0E0EBE22F
:100DF000F0E034E1220F8C9180FD216080818F77BB
:100E00008083832F8A95F1F7808180688083832F88
:100E10008A95F1F79F5F983069F7822F0895CF93F5
:100E2000DF93EC01ABE2B0E08C91886F8C938C91F6
:100E30008E7F8C93EAE2F0E08081896C80838081F0
:100E40008F7C8083E4E2F0E080818E7F8083E5E226
:100E5000F0E08081816080838C918F7B8C930E94F5
:100E6000F306282F30E0C901807F9070803491050F
:100E700009F040C020FF03C08D8188608D8321FF71
:100E800003C08D8182608D8322FF03C08D818160CC
:100E90008D8323FF03C08D8184608D830E94F306C0
:100EA000282F982F81FF03C08E8180618E8392FF4F
:100EB00003C08E8180628E8393FF03C08F81846024
:100EC0008F8394FF03C08F8188608F8395FF03C059
:100ED0008E8184608E8396FF03C08E8182608E83B4
:100EE00022231CF48E8181608E83EBE2F0E080810E
:100EF00080648083DF91CF910895DC01EAE2F0E025
:100F0000808186708083EBE2F0E08081896F80834E
:100F1000E4E2F0E08081807C8083E5E2F0E08081A3
:100F20008F638083E9E2F0E08081982F9170808167
:100F300083FD926080912F01981709F466C091306B
:100F4000F1F0913038F0923009F441C0933009F05B
:100F500051C029C0813041F415968C91159782605B
:100F600015968C93159746C0823009F043C01596AC
:100F70008C911597886015968C9315973BC083309C
:100F800041F415968C911597826015968C93159760
:100F900031C0882379F515968C9115978860159640
:100FA0008C93159727C0823041F415968C91159734
:100FB000826015968C9315971DC08130D9F41596D3
:100FC0008C911597886015968C93159713C088237C
:100FD00041F415968C911597826015968C93159710
:100FE00009C0833039F415968C9115978860159651
:100FF0008C93159790932F0183E080932E01159683
:101000008C911597809330010CC080912E0188231C
:1010100041F0815080932E018091300115968C9380
:1010200015974E9906C016968C9116978160169664
:101030008C930895EBE2F0E080818F7E808389E1DC
:1010400091E00197F1F789B190819061908381706F
:101050000895CF93DF93EC01E4E2F0E08081837C9C
:101060008083808182608083A5E2B0E08C918E6372
:101070008C93EAE2F0E080818E7F808380818061C2
:101080008083EBE2F0E08081816180838C918D7FB1
:101090008C931D9903C08D8181608D831C9903C041
:1010A0008D8184608D831B9903C08D8188608D83C1
:1010B0001A9903C08D8182608D830E941A0888234B
:1010C00019F48E8188608E830E941A08882319F48F
:1010D0008E8181608E830E941A08882319F48E8184
:1010E00084608E830E941A08882319F48E8182609E
:1010F0008E830E941A08882319F48E8180628E8361
:101100000E941A08882319F48E8180618E830E94C0
:101110001A08882319F48F8184608F83E5E2F0E058
:10112000808182608083DF91CF910895CF93DF9398
:10113000DC01E4E2F0E08081837C80838081826056
:101140008083E5E2F0E080818E638083EAE2F0E074
:10115000808180618083EBE2F0E080818F7E8083FC
:1011600092E02BE230E0E3E2F0E045E250E0E9011A
:1011700088818F7E88830000000080818C7309F451
:1011800057C0808185FD07C015968C9115978160A9
:1011900015968C931597808184FD07C015968C91C8
:1011A0001597826015968C931597808183FD07C0F3
:1011B00015968C911597846015968C931597808160
:1011C00082FD07C015968C911597886015968C93B3
:1011D0001597EA0188818D7F888300000000808157
:1011E00085FD07C016968C911697816016968C9394
:1011F0001697808184FD07C016968C9116978260A1
:1012000016968C931697808183FD07C017968C9154
:101210001797846017968C931797808182FD36C04C
:1012200017968C911797886017968C9317972EC0F6
:10123000EA0188818D7F888300000000808185FD20
:1012400007C016968C911697846016968C93169705
:10125000808184FD07C016968C911697886016963B
:101260008C931697808183FD07C016968C911697F4
:10127000806116968C931697808182FD07C0169622
:101280008C911697806216968C931697E901888147
:1012900080618883EA01888182608883915009F0A7
:1012A00066CFDF91CF91089590E020E0E5E2F0E095
:1012B00034E6A3E2B0E080818B7F8083832F8A9520
:1012C000F1F726958C9185FD20688081846080836C
:1012D000832F8A95F1F79F5F983069F7822F0895E1
:1012E000EF92FF920F931F937C0105E210E0F8014B
:1012F00080818C7E8083808184628083E4E2F0E060
:1013000080818F7D808380818C618083F8018081E2
:10131000886080838AEF8A95F1F70E945409F8016A
:101320008081877F80838AEAF70187831F910F91ED
:10133000FF90EF900895DC01EAE2F0E08081867092
:101340008083EBE2F0E08081896F8083E4E2F0E06B
:1013500080818E7F8083E5E2F0E080818160808300
:101360004E990CC016968C911697816016968C93A8
:10137000169704C09F5F9B3F21F4089590E0E3E23D
:10138000F0E0808180FDF6CF89B1982F892F80957C
:10139000282F217093FF226094FF246095FF28601E
:1013A00090E0E3E2F0E003C09F5F9B3F81F080812B
:1013B00080FFFACF89B180FF206183FF206284FF24
:1013C000206485FF20688FE7821B11968C93089517
:1013D000DC01EAE2F0E080818678808380818068A9
:1013E0008083EBE2F0E080818F7780838081896762
:1013F0008083E4E2F0E080818E7F8083E5E2F0E0AC
:1014000080818160808386E48A95F1F789B1807359
:1014100011F090E015C04E9907C016968C91169762
:10142000816016968C931697189B02C091E008C0B5
:1014300017968C911797886017968C93179791E061
:10144000EBE2F0E080818068808386E48A95F1F7A2
:10145000489907C015968C911597816015968C93C5
:1014600015974B9907C015968C9115978460159622
:101470008C9315974C9907C015968C911597886099
:1014800015968C9315974D9907C015968C911597C5
:10149000826015968C931597992391F44E9907C005
:1014A00016968C911697816016968C9316971899BC
:1014B00059C016968C911697826016968C9352C0DE
:1014C0004E9907C016968C911697826016968C934B
:1014D0001697189907C016968C91169784601696E1
:1014E0008C931697EBE2F0E080818F77808396E40F
:1014F000892F8A95F1F7808180688083892F8A956A
:10150000F1F780818F7780839A95F1F789B189739C
:1015100049F580818068808386E48A95F1F748994F
:1015200007C016968C911697806216968C93169724
:101530004B9907C016968C911697806116968C93DE
:1015400016974C9907C016968C9116978860169638
:101550008C9316974D9906C017968C9117978460B7
:1015600017968C93EBE2F0E0808180688083089589
:10157000DC01E4E2F0E08081817C8083E5E2F0E060
:1015800080818E638083E7E2F0E08081807C8083CD
:10159000E8E2F0E080818F638083EAE2F0E080811E
:1015A0008E7E8083EBE2F0E08081816180831D99F3
:1015B00007C017968C911797846017968C9317978E
:1015C0001C9907C016968C911697886016968C9376
:1015D00016971B9907C016968C91169782601696DF
:1015E0008C9316971A9907C015968C91159782605F
:1015F00015968C931597199907C015968C91159788
:10160000846015968C931597329907C017968C9124
:101610001797886017968C931797319907C016967D
:101620008C911697846016968C931697309906C005
:1016300016968C911697816016968C930895282F94
:10164000269511F437E009C037E0982F990F822FC3
:101650008170892B31502695C1F790E002C0880F28
:10166000991F3A95E2F7089589B1E5E2F0E090819B
:101670009E7F908328E7922F9A95F1F79081916051
:1016800090832A95F1F78295869587708095817071
:10169000089520E090E0A9E2B0E0E5E2F0E038E76C
:1016A00026958C9185FF206880818E7F8083832F93
:1016B0008A95F1F7808181608083832F8A95F1F785
:1016C0009F5F983069F7822F08950F931F93CF93F0
:1016D000DF93EC01EAE2F0E080818F7D8083ABE272
:1016E000B0E08C9180628C938081806880838C9143
:1016F00080688C93E4E2F0E0808181608083E5E2A1
:10170000F0E080818160808380EF8A95F1F78C9191
:101710008F778C9388E78A95F1F70E94490B182FF1
:101720000E94490B082F0E94490B982F11231CF48B
:101730008D8182608D83212F30E016FF03C08D8163
:1017400088608D8325FF03C08D8184608D8324FF95
:1017500003C08D8181608D83F901E870F07023FFF3
:1017600003C08F8188608F83B9016470707022FF1D
:1017700003C08F8184608F83892F8F70883009F038
:101780005AC0812F82958F70982F80FF03C08D8162
:1017900081608D8391FF03C08D8184608D8392FF72
:1017A00003C08D8188608D8393FF03C08D8182602B
:1017B0008D83802F8095482F4F70483008F040511E
:1017C000842F90E0880F991F880F991F909581951D
:1017D0009F4F8A83802F90E080959095807F9070B6
:1017E00095958795959587959595879595958795E1
:1017F000482F883008F04051842F90E0880F991FBF
:10180000880F991F909581959F4F8983EF2B19F031
:101810008F8188608F83672B19F08F8184608F831D
:1018200021FF03C08E8182608E8320FF6CC08E8179
:1018300081608E8368C0402F50E0CA01807C907028
:10184000803C9105D1F50F3F21F081E0809331017B
:101850000FC080913101882359F421FF03C08E818C
:1018600082608E8320FF4FC08E8181608E834BC04B
:1018700020FF02C08FE78C8321FF02C080E88B83AA
:1018800040FF02C08FE78B8341FF02C080E88C835A
:1018900042FF03C08E8180618E8343FF03C08E812F
:1018A00080628E8344FF03C08E8182608E8345FFF9
:1018B0002AC08E8181608E8326C0802F807F09F5AB
:1018C0001092310121FF03C08E8182608E8320FF40
:1018D00003C08E8181608E8340FF03C08E8188604B
:1018E0008E8341FF03C08E8184608E8342FF03C0DC
:1018F0008E8180618E8343FF06C08E8180628E83DD
:1019000002C010923101DF91CF911F910F91089584
:10191000382F8FE08A95F1F790E020E0E5E2F0E0E3
:101920004EE6A3E2B0E030FF04C080818061808396
:1019300003C080818F7E808380818B7F8083842F12
:101940008A95F1F726958C9185FD206880818460C9
:101950008083842F8A95F1F79F5F983011F0369538
:10196000E2CF8FE08A95F1F7822F0895CF92DF9230
:10197000FF920F931F93CF93DF93EC016B01E4E28F
:10198000F0E080818D7D808380818C618083E5E2C1
:10199000F0E080818E6380838081877F80838FE009
:1019A0008A95F1F781E00E94880C82E40E94880CFD
:1019B000082F10E0813409F411E0FF24033711F4FB
:1019C000FF24F394812F8F2990E020E030E003354D
:1019D00011F421E030E0822B932B892B09F483C092
:1019E0008FEF0E94880C8A3509F07DC08FEF0E942E
:1019F000880C282F982F80FD03C08F8184608F83EF
:101A000093FD03C08F8188608F831123A9F094FD1B
:101A100003C08D8181608D8396FD03C08D818460BC
:101A20008D8322231CF08D8188608D8395FD16C0E7
:101A30008D8182608D8312C0FF2081F091FD03C0F3
:101A40008F8181608F8392FD03C08F8182608F833D
:101A5000822F82958F7080958F708D838FEF0E947B
:101A6000880C282F982F82FD03C08E8180618E8381
:101A700093FD03C08E8180628E8390FD03C08E81B2
:101A800080648E8391FD03C08E8180688E8396FD75
:101A900003C08E8181608E8322231CF08E81826040
:101AA0008E8394FD03C08E8184608E8395FD03C078
:101AB0008E8188608E83FF2011F40335A1F48FEFAF
:101AC0000E94880C80588B838FEF0E94880C80586E
:101AD0008C838FEF0E94880C805889838FEF0E943F
:101AE000880C80588A830332D9F58FEF0E94880CC6
:101AF0008A35B1F58FEF0E94880C982F83FD03C0C3
:101B00008F8188608F83892F82958F7080958F70E9
:101B10008D838FEF0E94880C282F83FD03C08E8158
:101B200080628E8324FD03C08E8184608E8325FDB8
:101B300003C08E8188608E838FEF0E94880C80584E
:101B400089838FEF0E94880CF60180838FEF0E94BB
:101B5000880CF60182838FEF0E94880CF601848343
:101B6000E5E2F0E08081886080838FE08A95F1F77C
:101B7000DF91CF911F910F91FF90DF90CF9008954B
:101B800090E0E3E2F0E003C09F5F983C19F08081B1
:101B900081FDFACF089590E0E3E2F0E003C09F5F9B
:101BA000983C19F0808181FFFACF08950F931F931D
:101BB000CF93DF93EC01E4E2F0E080818D7C8083C1
:101BC00080818C608083E5E2F0E080818E63808399
:101BD000EAE2F0E080818E7E8083EBE2F0E08081BB
:101BE000816180838AE08A95F1F7489B5BC04C99BC
:101BF00003C08E8180648E83E5E2F0E08081877F80
:101C000080838AE08A95F1F71C9903C08D818160F9
:101C10008D831D9903C08D8184608D83489903C095
:101C20008D8188608D834C9903C08D8182608D8306
:101C3000E5E2F0E08081837F886080838AE08A9596
:101C4000F1F71C9903C08E8182608E831D9903C0B9
:101C50008E8184608E83489903C08E8181608E83DB
:101C60004C9903C08F8188608F83E5E2F0E080812A
:101C7000837F80838AE08A95F1F71C9903C08E8167
:101C800080628E831D9903C08E8180618E83489906
:101C900003C08E8188608E834C993EC18E8180689E
:101CA0008E833AC11C9B38C1E5E2F0E08081877FDA
:101CB000808380818B7F80830E94C00D1C991BC113
:101CC00005E210E0F8018081846080830E94CB0DE2
:101CD000F80180818B7F80830E94C00D1C9903C016
:101CE0008D8181608D831D9903C08D8184608D837A
:101CF000489903C08D8188608D834C9B02C010E0A1
:101D00001AC08D8182608D8310E015C08D81816045
:101D10008D831D9903C08D8184608D83489903C094
:101D20008D8188608D834C9B02C011E004C08D8141
:101D300082608D8311E0E5E2F0E080818460808341
:101D40000E94CB0D1C9903C08E8182608E831D99E9
:101D500003C08E8184608E83489903C08E81816028
:101D60008E834C9903C08F8188608F83E5E2F0E019
:101D700080818B7F80830E94C00D1C9903C08E815F
:101D800080628E831D9903C08E8180618E83489905
:101D900003C08E8188608E834C9903C08E818068D9
:101DA0008E83E5E2F0E08081846080830E94CB0D29
:101DB0004C9903C08E8180648E83E5E2F0E08081DF
:101DC0008B7F80830E94C00D1C9902C000E101C07E
:101DD00000E01D9B0062489B00644C9B0068E5E2AC
:101DE000F0E08081846080830E94CB0D1C9B0160A9
:101DF0001D9B0260489B04604C9B0860113019F4E5
:101E00008FE7801B8983E5E2F0E080818B7F808310
:101E10000E94C00D1C9902C000E101C000E01D9BA2
:101E20000062489B00644C9B0068E5E2F0E0808122
:101E3000846080830E94CB0D1C9B01601D9B02600F
:101E4000489B04604C9B0860113019F48FE7801B9D
:101E50008A83E5E2F0E080818B7F80830E94C00D61
:101E60001C9902C000E101C000E01D9B0062489B7C
:101E700000644C9B0068E5E2F0E080818460808330
:101E80000E94CB0D1C9B01601D9B0260489B04605F
:101E90004C9B0860113019F4802F80588C83E5E248
:101EA000F0E080818B7F80830E94C00D1C9902C06E
:101EB00000E101C000E01D9B0062489B00644C9B58
:101EC0000068E5E2F0E08081846080830E94CB0DB1
:101ED0001C9B01601D9B0260489B04604C9B08603A
:101EE000113019F4802F80588B83E5E2F0E0808177
:101EF0008C60808311C005E210E0F801808184606D
:101F000080830E94CB0DF80180818B7F80830E94AB
:101F1000C00D1C9BFBCEFDCEDF91CF911F910F9189
:101F20000895DC01E4E2F0E08081817C8083E5E2D9
:101F3000F0E080818E638083E7E2F0E08081827C44
:101F40008083808182608083E8E2F0E080818F631B
:101F5000808380818D7F808380818260808390E810
:101F60002FE0E3E2F0E0822F8A95F1F7808185FF90
:101F700003C011969C931197808184FF03C0129631
:101F80009C931297808183FF03C013969C931397B1
:101F9000808182FF03C014969C9314979F5F9F37A4
:101FA00011F711968C9111978E3719F411961C9296
:101FB000119712968C9112978E3719F412961C92E3
:101FC000129713968C9113978E3719F413961C92CF
:101FD000139714968C9114978E3719F414961C92BB
:101FE0001497309907C016968C91169781601696B3
:101FF0008C931697199907C016968C911697826044
:1020000016968C9316974C9907C016968C91169736
:10201000846016968C931697489906C016968C91F4
:102020001697886016968C930895E9E6F0E0808113
:1020300082608083EDE3F0E0808181608083AEE6A2
:10204000B1E08BE48C93E0EBF1E0808311978AE5BB
:102050008C933197808308951F93CF93DF93809162
:102060009501982F93500AF4A3C02091920180917A
:1020700091018D3209F09AC0983009F097C08CE038
:1020800090E0821B9109FC01E756FE4FEF0183ECC3
:10209000809362018AE58093000110923201808171
:1020A000807629F0CF010E941402982F76C0928189
:1020B00010926B018181882331F4ECE6F1E010820B
:1020C00092E0319766C0853031F49093960190E0AC
:1020D000EBE6F1E05EC08630D1F58381813041F4DA
:1020E00088E690E0909394018093930192E12BC055
:1020F000823041F48AE790E09093940180939301B9
:1021000090E221C08330F1F4992341F484EC90E013
:10211000909394018093930194E015C0913041F421
:1021200088EC90E090939401809393019AE20BC025
:10213000923041F482EF90E0909394018093930168
:102140009AE201C090E080E48093320126C088309A
:1021500021F491E0E8E9F1E01CC0893031F490937A
:10216000980190E0EBE6F1E014C08A3021F491E0B0
:10217000EBE6F1E00EC08B3021F090E0EBE6F1E011
:1021800008C08BE480936E018093B00190E0EBE691
:10219000F1E0F0939401E09393018F81882321F47F
:1021A0008E81891708F4982F909301011092950160
:1021B0008091000184FF57C0109101011F3F09F475
:1021C00052C0193008F05CC010920101E2E6F1E063
:1021D000808198E889278083112309F45DC02091CC
:1021E0009301309194018091320186FF14C0A3E6DF
:1021F000B1E080E090E0F901E80FF91FE491ED9380
:1022000001961817C1F7812F815090E00196F901CE
:10221000E80FF91F0FC0D901912FE3E6F1E08D918E
:1022200081939150E1F7812F815090E00196F9015F
:10223000E80FF91FF0939401E0939301193068F4CB
:1022400083E691E0612F0E949A11612F6C5F6C30E0
:1022500040F48FEF8093010104C08FEF8093010160
:102260006EE16093000194E1E9E2F0E08081867024
:10227000D1F49150D9F7109296011092900113C0A9
:10228000812F885080930101E2E6F1E0808198E897
:102290008927808318E0A3CF83E691E060E00E9465
:1022A0009A1164E0D6CFDF91CF911F9108951F93CB
:1022B000CF93DF93DC01162FEA01888184FF05C0EC
:1022C000898198E88927898302C08AE58883AE01DD
:1022D0004E5F5F4FFA01212F8D9181932150E1F7DD
:1022E000CA01612F0E949A11812F8C5F8883DF9130
:1022F000CF911F9108954FEA51E00E945711089520
:102300004DE651E00E9457110895A82FB92F80E0A3
:1023100090E041E050EA609530E009C02D918227BD
:102320009795879510F084279527305EC8F36F5FE7
:10233000A8F30895EADF8D939D930895CF93CFB7C7
:10234000CF93C395499BE9F7499B0BC0499B09C0B3
:10235000499B07C0499B05C0499B03C0499B01C0DD
:10236000C2C0C0919201DF93DD27C756DE4F2F9385
:102370002FEF499B03C02F91DF91E6CF0F931F935F
:102380004F936F9309B101FB20F93F933BE05F93BB
:102390001EC04E7F012F19B11670E1F021600000C0
:1023A0001DC0102F4D7F2260000009B1067091F012
:1023B0001DC04B7F2460012F000019B1167051F031
:1023C0001EC019B1167031F0477F28601BC019B1CB
:1023D000167009F462C04FEF297FD9F2012701FB83
:1023E00021F909B10670B1F3237FD9F2102711FB4F
:1023F00022F900C019B1167069F3277ED1F20127C6
:1024000001FB23F92F7CE9F209B1067019F31027BB
:1024100011FB24F92F7929F100C019B11670E9F1E7
:10242000012701FB25F92F7311F100C009B10670D6
:10243000A1F1102711FB26F92230F8F000C019B1E4
:10244000167059F1012701FB27F92430E0F04227EB
:10245000000009B14993102711FB20F93150C8F051
:10246000B6CF4F7E09B10670C1F02061D3CF206294
:1024700019B1167091F04F7DD6CF4F7B09B1067020
:1024800061F02064D9CF4F7719B1167031F0206810
:10249000DCCF11E01CBB002719C03B503195C31B9A
:1024A000D04011E01CBB0881033C09F10B34F9F06A
:1024B000209190011981110F1213EDCF4A81441F11
:1024C000093651F10D3211F0013E29F700939701C1
:1024D0005F913F916F914F911F910F912F91DF91DC
:1024E000CCB3C0FD2ECFCF91CFBFCF911895209107
:1024F0009701222369F3109195011123E1F53430FE
:10250000E2F13093950120939101109192013BE00B
:10251000311B3093920131C00091950101305CF57F
:102520000AE54F7049F43091000134FD27C0009353
:102530000001C2E6D1E026C0423049F030916D0181
:1025400034FD1CC000936D01CEE6D1E01BC030917C
:10255000AF0136FD13C00093AF01C0EBD1E012C054
:1025600005271127000019C0052711271FC00527BF
:102570001127000024C04AE502C032ED432FC4E118
:10258000D0E032E01AB11660599A0BB11AB956E090
:1025900020E866E020FF052727950BB917951C3F1B
:1025A000F8F66A95B9F720FF0527279500000BB9C3
:1025B00017951C3FC8F620FF05272795179566E05D
:1025C0001C3F0BB9A0F629913A9521F7097F10918C
:1025D0009601110F0BB9C651D04011F01093900124
:1025E00011E01CBB02601AB1197F402F497F53E0F4
:1025F0005A95F1F700C00BB91AB94BB969CF629F70
:10260000D001739FF001829FE00DF11D649FE00DEA
:10261000F11D929FF00D839FF00D749FF00D659F4B
:10262000F00D9927729FB00DE11DF91F639FB00D4A
:10263000E11DF91FBD01CF011124089597FB092E5B
:1026400005260ED057FD04D014D00AD0001C38F453
:1026500050954095309521953F4F4F4F5F4F0895CE
:10266000F6F790958095709561957F4F8F4F9F4FAE
:102670000895A1E21A2EAA1BBB1BFD010DC0AA1FC3
:10268000BB1FEE1FFF1FA217B307E407F50720F0DB
:10269000A21BB30BE40BF50B661F771F881F991F56
:1026A0001A9469F760957095809590959B01AC019F
:0A26B000BD01CF010895F894FFCF9B
:0226BA005AFFC5
:00000001FF
